:100000007828B400252084133230A6000030A700E1
:100010005D20A00AA50AA201A30100083405A600DC
:10002000640000083405A7002606270534060319D6
:10003000A20A0319A30A2708A600A4030319A5030B
:100040000319A00B10282208732884178004732832
:10005000A301A200FF30A207031CA307031C7328FF
:100060000330A100DF3036202A28A101E83EA0009D
:10007000A109FC30031C3F28A00703183C28A00757
:100080006400A10F3C2820184528A01C4928000026
:1000900049280800A20001304D28A80023082102A9
:1000A000031D5428220820020430031801300319CC
:1000B00002302805031DFF3073281030A800A1016D
:1000C000A001A70CA60C031C6B282208A00723087C
:1000D0000318230FA107A10CA00CA50CA40CA80BBE
:1000E0006128240873288313031383126400080013
:1000F00088308B00831667308F0083120730990099
:1001000085018316083085009F0183129F01051524
:10011000831605118312DC30A200FF30A3000530E6
:10012000840008300120B8002308B9003808A00076
:100130003908A100A30101304A20031D8728851436
:100140008316851083120516831605128312051176
:100150008316051183120730A300D0302920872889
:02400E00DC3C98
:00000001FF
